:103C00000C94221E0C943E1E0C943E1E0C943E1EE0
:103C10000C943E1E0C943E1E0C943E1E0C943E1EB4
:103C20000C943E1E0C943E1E0C943E1E0C943E1EA4
:103C30000C943E1E0C943E1E0C943E1E0C943E1E94
:103C40000C943E1E11241FBE20E0A89521BD20E04B
:103C500025BFEAE7FFE3A0E6B0E020E002C0059060
:103C60000D92A036B207D9F7A0E6B0E020E001C07F
:103C70001D92A036B207E1F70C94411E0C94401E31
:103C80001895CFE5D4E0DEBFCDBF8BE089B988E1E0
:103C90008AB9949A80B384FD38C10E94901F982FEE
:103CA000913609F42EC1913409F41AC1933609F4FE
:103CB00013C1933409F401C19E3609F422C19D3425
:103CC00009F4CEC0953609F4BAC09C3609F4B2C0E6
:103CD0009D3609F4A6C0903509F40FC19C3409F44F
:103CE0000CC1903709F499C0923509F488C0943416
:103CF00009F478C0943609F469C0963409F45EC0BA
:103D0000923709F457C09E3409F450C0943709F42F
:103D100046C0892F8857823018F40E94901FEDC04A
:103D20009435D9F3933529F19635E1F0963799F02A
:103D3000933739F09B3109F4B0CF8FE30E948A1F8B
:103D4000ACCF82E00E948A1F84E90E948A1F8EE124
:103D50000E948A1FA2CF81E30E948A1F80E30E94F3
:103D60008A1F9BCF82E30E948A1F83E30E948A1FDF
:103D700094CF81E40E948A1F86E50E948A1F82E513
:103D80000E948A1F82E40E948A1F8FE40E948A1F79
:103D90008FE40E948A1F84E50E948A1F7ECF86E6F8
:103DA0000E948A1F80E00E948A1F77CF69E083E02B
:103DB00090E007C069E081E090E003C069E080E046
:103DC00090E00E94A91F0E948A1F67CFCEBB8D2F53
:103DD00099278FBB21968CB381608CBB8DB30E94D9
:103DE0008A1F5BCFCEBB8D2F99278FBB21960E9458
:103DF000901F8DBBE29A8CB381FDFDCF7EC060E049
:103E0000CE010E94A91F8C01812F99270E948A1F31
:103E1000802F0E948A1F229640CF83E50E948A1F2E
:103E20003CCF65E0CE010E94961F61E1CE010E9469
:103E3000961F63C00E94901F0E94B41F5EC0C0E026
:103E4000D0E063E0CE010E94961F61E1CE010E94A6
:103E5000961FC058DF4F8CE3C030D80790F34DC099
:103E60000E94901FF82E6E01EE24EF14A0F40E9421
:103E7000901FB82E0B2D11270E94901F9927982F65
:103E80008827082B192BBE01C8010E949E1F22966D
:103E9000E394EF1460F38F2D0E948A1F8D2D9927D4
:103EA0000E948A1F8C2D0E948A1F8D2F99270E94A5
:103EB0008A1F8C2F0E948A1F20C00B2D11270E9461
:103EC000901F9927982F8827082B192BBE01C8010E
:103ED0000E949E1F229611C00E94901FB82E0DC0F6
:103EE0000E94901FC82FDD27DC2FCC270E94901F37
:103EF0009927C82BD92BCC0FDD1F8DE00E948A1F7C
:103F0000CCCE89E50E948A1FC8CE0E94000080E0C6
:103F100090E0FFCF8CB98BB186FFFDCF5E9A0895FC
:103F20008BB18823ECF78CB19927089525D0F92F10
:103F3000E82F67BFE895FFFF00001EC01DD0F72FD8
:103F4000E62F192E082E21E027BFE895FFFF00007D
:103F500013D012D0F92FE82F60FD67BFC895802DD0
:103F6000E395C895902D089507D0082E19E017BF46
:0A3F7000E895FFFF000000D008955F
:0400000300003C00BD
:00000001FF
